:020000040000FA
:1000000041EF07F0F76A140FF66E000EF7220900B1
:10001000F5501200000000000000005F0000000723
:10002000000700147F147F14242A7F2A1223130848
:10003000646236495522500005030000001C22412D
:10004000000041221C0014083E081408083E08085D
:100050000050300000080808080800606000002018
:10006000100804023E5149453E00427F4000426173
:100070005149462141454B311814127F10274545FF
:1000800045393C4A49493001710905033649494916
:1000900036064949291E0036360000005636000053
:1000A00008142241001414141414004122140802EC
:1000B00001510906324979413E7E1111117E7F4975
:1000C0004949363E414141227F4141221C7F4949F5
:1000D00049417F090909013E4149497A7F080808D9
:1000E0007F00417F41002040413F017F08142241B1
:1000F0007F404040407F020C027F7F0408107F3E1B
:100100004141413EF76A140FF66E010EF7220900D5
:10011000F55012007F090909063E4151215E7F0911
:10012000192946464949493101017F01013F4040B3
:10013000403F1F2040201F3F4038403F63140814B9
:100140006307087008076151494543007F4141003A
:1001500002040810200041417F0004020102044013
:1001600040404040000102040020545454787F482D
:100170004444383844444420384444487F38545434
:100180005418087E0901020C5252523E7F080404A2
:100190007800447D40002040443D007F102844000A
:1001A00000417F40007C041804787C0804047838FF
:1001B000444444387C14141408081414187C7C0833
:1001C0000404084854545420043F4440203C404018
:1001D000207C1C2040201C3C4030403C44281028FF
:1001E000440C5050503C4464544C44000836410088
:1001F00000007F0000004136080010080810087851
:1002000046414678F76A140FF66E020EF72209008F
:10021000F550120080E0F8FC3E0E0F070707070FAD
:100220001E7CF8F080FFFFFF0000000000000000CF
:10023000000000FFFFFF010F1F3F78F0E0E0E0E06B
:10024000E070783F1F07000000000070783CFEFF60
:10025000FF0000000000000000000000000000FFA0
:10026000FFFF0000000000000000000000E0E0E0F0
:10027000FFFFFFE0E0E0000000000030383C1E0E11
:10028000070707070F0EFEFCF8000000000080C003
:10029000E0F070383C1E0F0F03000000007CFFFFF1
:1002A000E3E1E0E0E0E0E0E0E0E0C0000000001CAE
:1002B0001E0E0E070707070F0EFEFCF000000000E1
:1002C0000000000C0E0E0E1E1F3777E3E1800000C9
:1002D0001C3C7C70F0E0E0E0E0E070783F1F0F0035
:1002E000000000000000C0E0F87C1EFFFFFF0000DF
:1002F0000000E0F0F8FEDFCFC3C1C0C0FFFFFFC0C9
:10030000C0C00001010101010101010101FFFFFF66
:1003100001010100F76A240FF66E030EF7220900AF
:10032000F55012000083FFFF7F8787C7C7C7C7C785
:10033000C787070300001F1F1F0F070301010101EB
:10034000010307FFFEF8001C3C7C70E0E0E0E0E009
:10035000F070783E1F0F0300000080E0F0783C1E34
:100360000F0703000000000000F8FFFF1F1D0C0E28
:100370000E0E0E0E1E3CFCF8E000071F3F7C70F0D6
:10038000E0E0E0E0F0707C3F1F0707070707070782
:10039000070707C7E7F77F3F1F0F030000000000B4
:1003A00080F0FCFF3F07010000000000000040F06B
:1003B000FE7F1F0300000000000000000000F0FCB2
:1003C000FC1E0F07070707078FFEFCF8000000C19F
:1003D000F3FF7F3F1E0E0E0E1F3F7BF9F0C00000A3
:1003E0000F3F7F78F0E0E0E0E0E0F0787F3F0F0043
:1003F000E0F8FC3E0E0F070707070F1E3EFCF8E073
:10040000000F1F3F7870F0E0E0E0E07070F8FFFF51
:100410001F000080C0C0E0E0E07078381E1F0703B6
:1004200000000000F76A340FF66E040EF722090090
:10043000F55012007072655F696E697431200A0DA3
:100440000000F76A520FF66E040EF7220900F5500D
:1004500012004C434400F76A660FF66E040EF72252
:100460000900F55012004272696768746E65737313
:100470000000F76A820FF66E040EF7220900F550AD
:10048000120041646A7573740000F76A9A0FF66E81
:10049000040EF7220900F5501200546563684465A4
:1004A0007369676E2E626500F76AB80FF66E040E08
:1004B000F7220900F5501200706F73745F696E695E
:1004C0007431200A0D00F76AD60FF66E040EF7227B
:1004D0000900F5501200566F703D20257520000070
:1004E000F76AF00FF66E040EF7220900F5501200BD
:1004F000202020202020202020202020202000003C
:10050000F76A100FF66E050EF7220900F55012007B
:100510002020202020200000F76A280FF66E050E0C
:10052000F7220900F55012002000F76A3A0FF66E24
:10053000050EF7220900F55012000A0A0D2A2A2A90
:100540002A2A2A2A2A2A2A2A2A2A2A203032352006
:100550002D20576972656C657373204D756C7469D5
:100560004D65746572205258202A2A2A2A2A2A2A7E
:100570002A2A2A2A2A2A2A200A0A0D00F76A8C0F18
:10058000F66E050EF7220900F5501200696E6974C7
:10059000204F4B200A0D0000F76AA80FF66E050EDB
:1005A000F7220900F550120020576972656C6573D7
:1005B0007320444D4D200A0D0000F76ACA0FF66EF5
:1005C000050EF7220900F550120020202000F76ADE
:1005D000DE0FF66E050EF7220900F55012004E6F81
:1005E000207369676E616C210000F76AFA0FF66E7E
:1005F000050EF7220900F55012002A202000F76AA4
:100600000E0FF66E060EF7220900F55012002A2A88
:100610002000F76A220FF66E060EF7220900F55049
:1006200012002A2A2A00F76A360FF66E060EF72203
:100630000900F55012003100F76A480FF66E060EF9
:10064000F7220900F5501200202020202020202031
:1006500020200000F76A640FF66E060EF7220900EC
:10066000F550120054582042617474657279206C00
:100670006F770000F76A840FF66E060EF722090006
:10068000F550120042757A7A65720000426A425053
:10069000C9DE000905E0422A9EA8FED7AD6EF7D755
:1006A000F2CF42F0F29EA96AA69CA69EA680A85010
:1006B00042BEF28E296E29507F0815E3C80E296EBE
:1006C000A96AA86EA69CA69EA684F2CF00F0F29E10
:1006D0000F01550EA76EAA0EA76EA682A6B2FED770
:1006E000A6940050F212000188EF07F0EA6A420E69
:1006F000E96EEF500FE0010E016E006A002EFED78A
:10070000012EFBD74A0E006E002EFED7000000001F
:10071000EF2EF1D7000C080E4A6E4A520DE081967A
:100720004950800B02E1819801D0818800008186C8
:10073000D89049364A06F1D7000C819A819C48C06E
:1007400049F0E9DF818C000C4650070B4009476EE9
:10075000486EF3DF45507F0B8009476E486EEDDF32
:10076000000C818A819C45C049F0D5DF818C000C4A
:10077000456A466AE9DF010E2B6EF80E2A6E2A5290
:1007800002E12B5207E0456AECDF2A50D8B42B0671
:100790002A06F5D7E3EF03F0818A818C819E0A0E49
:1007A000426EA4DF818E210E486EC7DF29C048F05B
:1007B000C4DF130E486EC1DF200E486EBEDF090E87
:1007C000486EBBDFD5D7080E486EB7DF0C0E486EFB
:1007D000B4DF000C26501F0801E335D026507F08F7
:1007E00001E231D0256A255004082BE326504F083A
:1007F00011E32650E00F050DF3CF27F025502724F5
:10080000036AF2CF46F0F29E02EC00F046BEF28E92
:10081000286E12D026504F080FE22650B00F050D5B
:10082000F3CF27F025502724036AF2CF46F0F29E3B
:1008300069DC46BEF28E286E28C045F092DF252A7C
:10084000D2D7456A8EDF28EF04F044C026F0C2D725
:10085000000C4650016A455C03E245C000F00CD034
:10086000006A080E476E453600364650005CD8B028
:10087000006E0136472EF7D7000C015043C045F0FB
:10088000640E466EE6DF00C043F00150300E07E113
:1008900044A20DD044B60BD044B8200E03D04496E9
:1008A00044984480012601509EA8FED7AD6E43C0F7
:1008B00045F00A0E466ECDDF00C043F00150300E09
:1008C00006E144B609D044A007D044B8200E012662
:1008D00001509EA8FED7AD6E300E432643509EA811
:1008E000FED7AD6ED7EF04F01E0E456E010E466EBC
:1008F0002BDF426A4250A5DD000904E0422A446E23
:10090000A4DFF8D70C0E456E020E466E1DDF426A5C
:100910004250A1DD000904E0422A446E96DFF8D778
:10092000180E456E030E466E0FDF426A4250A1DD7F
:10093000000904E0422A446E88DFF8D7030E456EB2
:10094000050E466E01DF426A42509FDD000904E059
:10095000422A446E7ADFF8D7426A4250A5DD000988
:1009600005E0422A9EA8FED7AD6EF7D781A424D019
:10097000293C01D021D0010E2926C80E426EB6DED8
:10098000210E486EDADE29C048F0D7DE426A4250B6
:100990009ADD422A006E00509EA8FED7AD6E050E6D
:1009A000425CF5E129C043F01B0E446E66D7200E71
:1009B0009EA8FED7AD6EDAD7293C03D0800E296EF3
:1009C000CBD7A96A29C0A8FFA69CA69EA684F2CF71
:1009D00000F0F29E0F01550EA76EAA0EA76EA6821A
:1009E000A6B2FED7A6940050F2120001D5DE8AEF1F
:1009F00007F00A941B6A1A6A196A186A1F6A1E6A43
:100A00001D6A1C6A81A209D0010E1826D8B0192AC5
:100A1000D8B41A2AD8B41B2AF5D71B5207E11A52A8
:100A200005E1195203E1185014080AE21B5208E1CB
:100A30001A5206E1195204E118501F0801E301D0CF
:100A400066D081B209D0010E1C26D8B01D2AD8B4B8
:100A50001E2AD8B41F2AF5D71F5207E11E5205E1FE
:100A60001D5203E11C5019080AE21F5208E11E52F0
:100A700006E11D5204E11C50270801E301D047D0D4
:100A80001B6A1A6A196A186A1F6A1E6A1D6A1C6A3A
:100A900081A209D0010E1826D8B0192AD8B41A2A72
:100AA000D8B41B2AF5D71B5207E11A5205E1195297
:100AB00003E1185014080AE21B5208E11A5206E139
:100AC000195204E118501F0801E301D020D081B26F
:100AD00009D0010E1C26D8B01D2AD8B41E2AD8B4BD
:100AE0001F2AF5D71F5207E11E5205E11D5203E1EF
:100AF0001C5019080BE21F5209E11E5207E11D525A
:100B000005E11C50270802E30A8401D000D019EF48
:100B100006F00A921B6A1A6A196A186A1F6A1E6A24
:100B20001D6A1C6A81A209D0010E1826D8B0192AA4
:100B3000D8B41A2AD8B41B2AF5D71B5207E11A5287
:100B400005E1195203E1185019080BE21B5209E1A3
:100B50001A5207E1195205E118502A0802E30A82E5
:100B600001D002D081A2FED72FEF06F01B6A1A6ACD
:100B7000196A186A1F6A1E6A1D6A1C6A81A209D056
:100B8000010E1826D8B0192AD8B41A2AD8B41B2AAC
:100B9000F5D71B5207E11A5205E1195203E118502B
:100BA0000D080BE21B5209E11A5207E1195205E147
:100BB0001850160802E30A8015D01B5207E11A529A
:100BC00005E1195203E1185004080BE21B5209E138
:100BD0001A5207E1195205E118500D0802E30A9074
:100BE00001D002D081A2FED7FCEF05F0106A080EFA
:100BF0000F6E0F520AE0BAD70AB010800F500108EA
:100C000002E2D89010360F06F4D735EF06F0116ADD
:100C1000126A136A7F0E066E06BE15D006500008D3
:100C200012E27F0E056E05BE09D00550000806E2EF
:100C3000E0D60AA401D00CD00506F5D70AA401D04D
:100C400007D00606E9D70AB403D0020E116E4AD0C7
:100C5000076A07BE03D00750090812E35AD70AB241
:100C600003D0030E116E3ED0C1D7036A0750420F66
:100C7000E96E000E0320EA6E10C0EFFF072AE9D7E5
:100C8000040E116E4250AA0803E1030E126E03D047
:100C9000010E126E27D04350A50803E1030E126E19
:100CA00003D0020E126E1ED04A50CC0803E1030E90
:100CB000136E03D0010E136E15D04B50AA0803E13A
:100CC000030E136E03D0020E136E0CD0050E116EC0
:100CD00044C021F045C022F046C023F047C024F0B4
:100CE00048C020F0A5EF07F0456A42C046F02CDD71
:100CF000436A435070EC02F0000904E0432A446E5A
:100D0000A4DDF7D7000C43BE10D00F0E006E4238A2
:100D100000160A0E005C03E2300E002602D043509B
:100D2000002600509EA8FED7AD6E0F0E42160A0E8A
:100D3000425C02E2300E02D0439E435042264250B3
:100D40009EA8FED7AD6E000C44502F0802E379D068
:100D500004D04450390801E274D0415203E1070E37
:100D6000416E17D04150070803E11B0E416E11D0B0
:100D700041501B0803E12F0E416E0BD041502F084C
:100D800003E1430E416E05D04150430802E1070ED6
:100D9000416E256A2550320854E3445030080FE173
:100DA000300E445C330DF3502524036AF2CF47F034
:100DB000F29E02EC01F047BEF28E286E25D0445020
:100DC000340810E3300E445C330DF3502524010F3A
:100DD000036AF2CF48F0F29E02EC01F048BEF28EB8
:100DE000286E12D0445034080FE2300E445C330DAC
:100DF000F3502524010F036AF2CF48F0F29E8AECEB
:100E000001F048BEF28E286E255205E141C045F042
:100E1000466A9ADC11D02550110806E141C045F020
:100E2000010E466E91DC08D02550220805E141C034
:100E300045F0020E466E88DC28C045F092DC252A7B
:100E4000A9D7000C43BE0FD00F0E006E423800161B
:100E50000A0E005C03E2300E002602D0435000264A
:100E600000C044F071DF0F0E42160A0E425C02E22F
:100E7000300E02D0439E4350422642C044F064DF0D
:100E8000000CF86AD09EFE0E006E080E016E020E77
:100E9000E96E000EEA6EEF6AE92AD8B4EA2A002E5B
:100EA000FAD7012EF8D7EA6AE96AB8960C0EAF6E47
:100EB000260EAC6E900EAB6EC150C00B0F09C16E0A
:100EC000070EB46E0F0E926E060E936E910E946E18
:100ED0008088C29094928B92B70EB11694928B92A6
:100EE0000C0EBA6E000E0609CA6E1A0ECB6E0D0EEF
:100EF000BB6E930E946E426A425095EC02F000096C
:100F000005E0422A9EA8FED7AD6EF6D746EF03F065
:100F100043DCEAD4426A4250BEEC02F0000905E02C
:100F2000422A9EA8FED7AD6EF6D7456A050E466EDC
:100F30000BDC426A4250CCEC02F0000904E0422A89
:100F4000446E83DCF7D7809862D6808811500208FF
:100F500024E1040E426EC8DE456A030E466EA4EC20
:100F600003F0426A4250DDEC02F0000904E0422A3C
:100F7000446E6BDCF7D70C0E456E040E466EA4EC87
:100F800003F0426A4250E7EC02F0000904E0422A12
:100F9000446E5BDCF7D7D7D743D01150030814E178
:100FA000040E426EA1DE456A030E466EA4EC03F009
:100FB000426A4250F5EC02F0000904E0422A446E15
:100FC00044DCF7D7C0D72CD01150040814E1040E2C
:100FD000426E8ADE456A030E466EA4EC03F0426A56
:100FE0004250FFEC02F0000904E0422A446E2DDC7E
:100FF000F7D7A9D715D01150050812E1040E426E9B
:1010000073DE456A030E466EA4EC03F0426A42505A
:1010100009EC03F0000904E0422A446E16DCF7D71D
:10102000456A050E466EA4EC03F03D0E9EA8FED761
:10103000AD6E200E9EA8FED7AD6E21C042F0D70E39
:10104000436E61DE22C042F0D70E436E5CDE23C0E9
:1010500042F0D70E436E57DE24C042F0D70E436EE7
:1010600052DE200E9EA8FED7AD6E0A0E9EA8FED7B9
:10107000AD6E0D0E9EA8FED7AD6E456A466AA4EC15
:1010800003F0416A212C0BD0426A425013EC03F06A
:10109000000904E0422A446E57DEF7D734D0060E2A
:1010A000456E466AA4EC03F0426A4250DDEC02F061
:1010B000000905E0422A446E25EC04F0F6D7060E3E
:1010C000456E010E466EA4EC03F0426A4250DDEC20
:1010D00002F0000905E0422A446E25EC04F0F6D740
:1010E000060E456E020E466EA4EC03F0426A4250B4
:1010F000DDEC02F0000905E0422A446E25EC04F024
:10110000F6D7070E416E22500F0833E1180E456ED8
:10111000466AA4EC03F0426A42501CEC03F000095A
:1011200005E0422A446E25EC04F0F6D7180E456E11
:10113000010E466EA4EC03F0426A42501CEC03F030
:10114000000905E0422A446E25EC04F0F6D7180E9B
:10115000456E020E466EA4EC03F0426A42501CEC4F
:1011600003F0000905E0422A446E25EC04F0F6D7AE
:101170000FD022C042F0D70E436E64DE23C042F08F
:10118000D70E436E5FDE24C042F0D70E436E5ADEA8
:1011900020A81ED0456A010E466EA4EC03F0180E7E
:1011A000456EB1EC03F0180E456EB1EC03F0180E6D
:1011B000456EB1EC03F0180E456EB1EC03F0180E5D
:1011C000456EB1EC03F0180E456EB1EC03F010D093
:1011D000456A010E466EA4EC03F0426A42508CEC64
:1011E00002F0000905E0422A446E25EC04F0F6D72F
:1011F00020A60FD02D0E456E020E466EA4EC03F015
:10120000C00E456EB1EC03F0C00E456EB1EC03F0BC
:101210000CD02D0E456E020E466EA4EC03F0456A0E
:10122000B1EC03F0456AB1EC03F020A40FD03F0EFF
:10123000456E020E466EA4EC03F0C00E456EB1EC96
:1012400003F0C00E456EB1EC03F00CD03F0E456EBE
:10125000020E466EA4EC03F0456AB1EC03F0456A59
:10126000B1EC03F020A211D0456A050E466EA4EC45
:1012700003F0426A42502AEC03F0000905E0422ADA
:10128000446E25EC04F0F6D708D0456A050E466E8C
:10129000A4EC03F0050E426E27DD20A014D0300E22
:1012A000456E040E466EA4EC03F0426A42503AECDE
:1012B00003F0000905E0422A446E25EC04F0F6D75D
:1012C000910E946E13D0300E456E040E466EA4EC53
:1012D00003F0426A425080EC02F0000905E0422A25
:1012E000446E25EC04F0F6D7930E946E2CD60300D2
:00000001FF
